:100000000C9434000C9451000C9451000C94510049
:100010000C9451000C9451000C9451000C9431013B
:100020000C9451000C9451000C9451000C9400015C
:100030000C9451000C9451000C94CF000C9451007E
:100040000C9451000C9451000C9451000C945100EC
:100050000C9451000C9451000C9451000C945100DC
:100060000C9451000C94510011241FBECFEFD8E026
:10007000DEBFCDBF11E0A0E0B1E0E4E4F7E002C0F4
:1000800005900D92A832B107D9F711E0A8E2B1E0CE
:1000900001C01D92AD32B107E1F70E948B010C94B3
:1000A000A0030C9400000F931F93CF93DF93EC01F8
:1000B00080917C00857E846080937C0080917A00B2
:1000C000806480937A0080917A0086FDFCCF6091F5
:1000D00078007091790080E090E00E94870220E033
:1000E00030E040E854E40E94190320E030EC4FE790
:1000F00054E40E941F026C837D838E839F8301E002
:1001000010E02A893B894C895D890E94150387FF8D
:1001100002C000E010E0198B088B8EA19FA18230F5
:10012000910561F08330910599F00197C9F416BCEF
:1001300080916E00826080936E0016C010928500E0
:100140001092840080916F00826080936F000CC0D9
:100150001092B2008091700082608093700004C0A1
:1001600081E090E00E94A00378949FB7F89480917A
:100170002A019FBF8823C9F310922A01EAA1FBA19B
:1001800088899989892B19F08081886002C08081D3
:10019000877F8083DF91CF911F910F9108951F92E8
:1001A0000F920FB60F9211242F933F938F939F932B
:1001B00080912801909129010196909329018093C3
:1001C000280180912A01813091F0209128013091FD
:1001D000290180912B0190912C012817390738F0C3
:1001E00081E080932A0110922901109228019F91A9
:1001F0008F913F912F910F900FBE0F901F901895E8
:100200001F920F920FB60F9211242F933F938F934B
:100210009F93809128019091290101969093290143
:100220008093280180912A01813091F0209128014A
:100230003091290180912B0190912C0128173907C9
:1002400038F081E080932A01109229011092280150
:100250009F918F913F912F910F900FBE0F901F9004
:1002600018951F920F920FB60F9211242F933F9360
:100270008F939F93809128019091290101969093EB
:1002800029018093280180912A01813091F02091E9
:1002900028013091290180912B0190912C01281780
:1002A000390738F081E080932A01109229011092D9
:1002B00028019F918F913F912F910F900FBE0F902A
:1002C0001F901895FC01539A8BE290E093A382A3B0
:1002D00085B5836085BD21E030E035A324A38AE0A5
:1002E00090E090932C0180932B0184B5826084BDB3
:1002F00089EF87BD37A326A3ACE7B0E08C91806C73
:100300008C93AAE7B0E08C9187688C9311A210A21D
:1003100080E090E00895CF92DF92EF92FF9280E02C
:1003200091E00E946201C12CD12C760160E070E066
:10033000CB016093000170930101809302019093BF
:10034000030180E091E00E9453008FEFC81AD80AA1
:10035000E80AF80AC701B6010E9487022FE632E1D7
:1003600043E05BE30E94190320E030E0A9010E9412
:10037000BB01DFCF5058BB27AA270ED01CC10DD11F
:1003800030F012D120F031F49F3F11F41EF402C17D
:100390000EF4E095E7FBF8C0E92F1ED180F3BA1701
:1003A000620773078407950718F071F49EF536C14C
:1003B0000EF4E0950B2EBA2FA02D0B01B901900180
:1003C0000C01CA01A0011124FF27591B99F0593FC4
:1003D00050F4503E68F11A16F040A22F232F342F0C
:1003E0004427585FF3CF469537952795A795F0405A
:1003F0005395C9F77EF41F16BA0B620B730B840B6F
:10040000BAF09150A1F0FF0FBB1F661F771F881F26
:10041000C2F70EC0BA0F621F731F841F48F487957E
:1004200077956795B795F7959E3F08F0B3CF93956D
:10043000880F08F09927EE0F9795879508950CD0AF
:10044000BAC0B2D040F0A9D030F021F45F3F19F02B
:100450009BC05111E4C09EC0BFD098F39923C9F34B
:100460005523B1F3951B550BBB27AA2762177307BA
:10047000840738F09F5F5F4F220F331F441FAA1F6E
:10048000A9F333D00E2E3AF0E0E830D0915050402E
:10049000E695001CCAF729D0FE2F27D0660F771FDC
:1004A000881FBB1F261737074807AB07B0E809F0BE
:1004B000BB0B802DBF01FF2793585F4F2AF09E3F53
:1004C000510568F061C0ABC05F3FECF3983EDCF3D0
:1004D000869577956795B795F7959F5FC9F7880FCC
:1004E000911D9695879597F90895E1E0660F771F1E
:1004F000881FBB1F621773078407BA0720F0621BAF
:10050000730B840BBA0BEE1F88F7E0950895E894FF
:1005100009C097FB3EF490958095709561957F4F4B
:100520008F4F9F4F9923A9F0F92F96E9BB279395F9
:10053000F695879577956795B795F111F8CFFAF409
:10054000BB0F11F460FF1BC06F5F7F4F8F4F9F4F3A
:1005500016C0882311F096E911C0772321F09EE898
:10056000872F762F05C0662371F096E8862F70E0FE
:1005700060E02AF09A95660F771F881FDAF7880FD8
:100580009695879597F9089597F99F6780E870E0A9
:1005900060E008959FEF80EC089500240A941616F9
:1005A000170618060906089500240A941216130661
:1005B000140605060895092E0394000C11F48823EF
:1005C00052F0BB0F40F4BF2B11F460FF04C06F5F0B
:1005D0007F4F8F4F9F4F089557FD9058440F551FE1
:1005E00059F05F3F71F04795880F97FB991F61F0B5
:1005F0009F3F79F087950895121613061406551F2C
:10060000F2CF4695F1DF08C0161617061806991F97
:10061000F1CF86957105610508940895E894BB278C
:1006200066277727CB0197F9089566D008F48FEFF6
:1006300008950BD0C0CFB1DF28F0B6DF18F09523B6
:1006400009F0A2CFA7CF1124EACFC6DFA0F3959F70
:10065000D1F3950F50E0551F629FF001729FBB27A9
:10066000F00DB11D639FAA27F00DB11DAA1F649F55
:100670006627B00DA11D661F829F2227B00DA11D08
:10068000621F739FB00DA11D621F839FA00D611D8E
:10069000221F749F3327A00D611D231F849F600DAF
:1006A000211D822F762F6A2F11249F5750408AF0E8
:1006B000E1F088234AF0EE0FFF1FBB1F661F771F74
:1006C000881F91505040A9F79E3F510570F05CCFB4
:1006D000A6CF5F3FECF3983EDCF386957795679560
:1006E000B795F795E7959F5FC1F7FE2B880F911D92
:1006F0009695879597F90895990F0008550FAA0BBD
:10070000E0E8FEEF16161706E807F907C0F0121624
:100710001306E407F50798F0621B730B840B950B27
:1007200039F40A2661F0232B242B252B21F408957C
:100730000A2609F4A140A6958FEF811D811D089519
:04074000F894FFCF5B
:1007440000000000000000000000000000000000A5
:10075400000000002F440AD7233C020001000000DF
:0807640000000000000000008D
:00000001FF
